S123C0007EC34E7E7FE87EC6107EC61A7EC62A7EC6267EC6447EC6427EC64B7EC6667EC693
S123C0207A7EC6217EC6460D0A040D0A3E20040D0A0A4D4333206D6F6E69746F7220312E74
S123C040330D0A44616E69656C20547566766573736F6E20323031332D323031340D0A0D5A
S123C0600A20472020476F2028525449290D0A204A20204A756D7020746F20616464726575
S123C08073730D0A204C20204C6F6164205331392066726F6D20636F6E736F6C650D0A2078
S123C0A04D43204D656D6F7279206368616E67650D0A204D44204D656D6F72792064756D06
S123C0C0700D0A205252205072696E7420636F6E74656E7473206F6620737461636B0D0A14
S123C0E020525320526573657420737461636B20706F696E7465720D0A2052432043686105
S123C1006E676520737461636B2043430D0A205241204368616E676520737461636B20413E
S123C1200D0A205242204368616E676520737461636B20420D0A205258204368616E6765EB
S123C14020737461636B20580D0A205250204368616E676520737461636B2050430D0A20CE
S123C16050202053656C65637420492F4F20706167650D0A20582020456E7465722065785D
S123C18074656E64656420524F4D0D0A040D0A4343204220204120205820202020504320B3
S123C1A0202053502020202020482049204E205A205620430D0A040D0A41444452202030C9
S123C1C020203120203220203320203420203520203620203720202038202039202041207D
S123C1E020422020432020442020452020460D0A040D0A4C6F616420533139207265636F6F
S123C20072640D0A040D0A0A4C6F6164206661696C202D205072657373205920746F206353
S123C2206F6E74696E75650D0A040D0A4C6F6164204F4B0D0A040D0A54524150206174200E
S123C240616464726573733A2024040D0A506172616D65746572206572726F720D0A048EC7
S123C2607F00BF7F08BDC6B0BDC5D486FF9700868797024F9714CEC02ABDC61ABDC6108147
S123C2800D27F384DF814826037EC332814726037EC33B814A26037EC33F815226037EC28E
S123C2A0ED814D26037EC2C4814C26037EC528815026037EC5B2815826037ED000863FBD70
S123C2C07FE820B2BDC610810D26037EC27684DF814326037EC40D814626037EC44F81443C
S123C2E026037EC49D863FBD7FE87EC276BDC610810D26037EC27684DF815226037EC3549F
S123C300814126037EC39E814226037EC3B0815826037EC3C2815026037EC3DA814326036B
S123C3207EC3F2815326037EC404863FBD7FE87EC276CEC02FBDC61A7EC276BE7F083B86CE
S123C34020BD7FE8BDC67A24036E007EC276BF7F087EC276CEC18DBDC61AFE7F0808BDC688
S123C36044BDC644BDC644BDC642BDC642CE7F08BDC6428620BD7FE8FE7F0808E600CE0038
S123C3800658588620BD7FE85825088630BD7FE87EC3988631BD7FE80926E87EC276863D76
S123C3A0BD7FE8FE7F08BDC6662402A7037EC276863DBD7FE8FE7F08BDC6662402A7027EBF
S123C3C0C276863DBD7FE8BDC67A240BFF7F0CFE7F08FC7F0CED047EC276863DBD7FE8BD2D
S123C3E0C67A240BFF7F0CFE7F08FC7F0CED067EC276863DBD7FE8FE7F08BDC6662402A769
S123C400017EC2768E7F00BF7F087EC2768620BD7FE8BDC67A242FCEC027BDC61ACE7F0C93
S123C420BDC642FE7F0CBDC644FF7F0CBDC666240E09A700A10027DF863FBD7FE820D88185
S123C440DD27D47EC276CEC24BBDC61A7EC2768620BD7FE8BDC67A2432FF7F0E862DBD7F84
S123C460E8BDC67A2425FF7F0CBC7F0E231D08FF7F0C8620BD7FE8BDC666240F16FE7F0E5E
S123C480E70008BC7F0C26F87EC276CEC24BBDC61A7EC276CEC24BBDC61A7EC2768620BDCF
S123C4A07FE8BDC67A24EDFF7F0CCEC027BDC61AB67F0D84F0B77F0DCEC1B7BDC61A8610B5
S123C4C0B77F0BCE7F0CBDC6428620BD7FE8FE7F0CFF7F0EBDC644FF7F0CB67F0D840F8173
S123C4E00826058620BD7FE8810026E8FE7F0EFF7F0C8620BD7FE8A600817E220481202C35
S123C50002862EBD7FE808FF7F0CB67F0D840F26E6CEC027BDC61A7A7F0B270220A5BDC603
S123C52010810D278B7EC276CEC1F1BDC61A860DBD7FE88639B77FE8BDC610815326F4BD02
S123C540C61081392757813126E97F7F0ABDC66616FB7F0AF77F0A8002B77F0BBDC67A2419
S123C56025F67F0AFB7F0CFB7F0DF77F0ABDC66616FB7F0AF77F0A7A7F0B2705A700082084
S123C580EC7C7F0A27A8867EB77FE8CEC205BDC61ABD7FEB84DF815926F77EC276BDC610B9
S123C5A0810D26F9867EB77FE8CEC22ABDC61A7EC276863DBD7FE886FF9700BDC64B2404A2
S123C5C081072309CEC24BBDC61A7EC2768A8097027EC27686059710860A9711961239379A
S123C5E0D61158585824F9971333399612961184C0810027F8814027F296123996129611D8
S123C60084C081002707814027F2860139860039BD7FEB7E7FE8BD7FE808A600810426F64B
S123C62039CEC02720F444444444840F8B30813923028B077E7FE8A600BDC626A600087EC5
S123C640C62A8DF38DF186207E7FE8BDC61080302B1281092F0C84DF81112B0881162E0427
S123C66080070D390C39BDC64B240D4848484816BDC64B24031B0D390C398DEA240DB77FF6
S123C6800C8DE32406B77F0DFE7F0C39BF7F08BDC3547EC276BF7F08CEC236BDC61AFE7FF5
S123C6A008C6063ABDC642CEC027BDC61A7EC276867ECEC276B77FFDFF7FFECEC68CB77F8C
S123C6C0FAFF7FFBCEC33BB77FF7FF7FF8CEC33BB77FF4FF7FF5CEC33BB77FF1FF7FF2CEDA
S123C6E0C33BB77FEEFF7FEFCEC5DFB77FE8FF7FE9CEC5EDB77FEBFF7FECCEC5FEB77FE5F9
S107C700FF7FE63994
S105FFEEC695B2
S111FFF27FEE7FF17FF47FF77FFA7FFDC25F21
S9030000FC
